:100000000C9446000C9463000C9463000C94630001
:100010000C9463000C9463000C9463000C946300D4
:100020000C9463000C9463000C9463000C946300C4
:100030000C9463000C9463000C9463000C946300B4
:100040000C9463000C9463000C9463000C946300A4
:100050000C9463000C9463000C9463000C94630094
:100060000C9463000C9463000C9463000C94630084
:100070000C9463000C9463000C9463000C94630074
:100080000C9463000C9463000C94630011241FBE55
:10009000CFEFD0E1DEBFCDBF11E0A0E0B1E0ECEBEF
:1000A000F2E000E00BBF02C007900D92A030B10754
:1000B000D9F711E0A0E0B1E001C01D92A030B10776
:1000C000E1F70C94CF000C940000CF93DF93CDB7F1
:1000D000DEB7F8948FEF80933A008FEF80933B0068
:1000E00083EE80933700109238007894DF91CF919F
:1000F0000895CF93DF93CDB7DEB721970FB6F8946D
:10010000DEBF0FBECDBF198282E00E94340188237A
:1001100019F089818160898383E00E9434018823FA
:1001200019F089818260898384E00E9434018823E8
:1001300019F08981846089834FEF60E089810E9492
:10014000D90021960FB6F894DEBF0FBECDBFDF9168
:10015000CF910895CF93DF93CDB7DEB782E00E94B1
:100160003401682F80E00E94F70083E00E94340190
:10017000682F81E00E94F70084E00E943401682F1C
:1001800082E00E94F700DF91CF910895CF93DF9333
:10019000CDB7DEB70E9465000E94AA00FDCFCFEF69
:1001A000D0E1DEBFCDBF0E94C60080E090E00C949D
:1001B0005D01CF93DF93CDB7DEB723970FB6F894E9
:1001C000DEBF0FBECDBF89836A834B838B818F3F98
:1001D00029F48FEF9981891B80933B0023960FB6FA
:1001E000F894DEBF0FBECDBFDF91CF910895CF93BE
:1001F000DF93CDB7DEB724970FB6F894DEBF0FBEFE
:10020000CDBF89836A8380913B008B838A818F3F36
:1002100091F48981282F332781E090E0022E02C0DB
:10022000880F991F0A94E2F780958C839B818C81BB
:1002300089238B830DC08981282F332781E090E0AB
:1002400002C0880F991F2A95E2F72B81822B8B839E
:100250008B8180933B0024960FB6F894DEBF0FBECF
:10026000CDBFDF91CF910895CF93DF93CDB7DEB7A8
:1002700022970FB6F894DEBF0FBECDBF89831A82D6
:1002800080913600282F33278981992702C0359520
:1002900027958A95E2F7C90181709070009711F057
:1002A0008FEF8A838A81992722960FB6F894DEBF52
:0C02B0000FBECDBFDF91CF910895FFCFAE
:00000001FF
